:0600000022C0FECFFDCF7F
:10000600FCCFFBCFFACFF9CFF8CFF7CF5DC0F5CF56
:10001600F4CFF3CFF2CFF1CFF0CFEFCF1027E80335
:1000260064000A0001000010000110000100000039
:1000360000000000000000000A0004003400000078
:10004600F894EE27ECBBF1E0FBBFEBBFE5BFE6BFE4
:100056008DE0A2E0BB27ED938A95E9F780E092E078
:10006600A0E6ED930197E9F7EEE3F0E0859195912F
:10007600009761F0A591B59105901590BF01F0012B
:1000860005900D920197E1F7FB01F0CFEFE5EDBF8B
:10009600E2E0EEBFC0EED0E01CC1AA935D9BFECFAE
:1000A600E881ECB921960895BA93AA93E981F07094
:1000B600EBBB939A9398E881EBBBE981F070E8BBC0
:1000C600E881EBBB229608950A921A92FA926A93F5
:1000D6007A938A939A93AA93BA93EA93FA93EFB789
:1000E600EA9384D11BB10CB1DD24E12FEC7109F048
:1000F600E0C0F20131962F013197E052FF4F0083A5
:10010600E7E0F1E0E415F50509F0D3C044245524F1
:100116000091E000E02FF0E0E33CA0E0FA0761F494
:10012600CC24A9ECBADFA8E1B8DFA0E1B6DFA8E0ED
:10013600B4DFA1E1B2DFBDC0E43CA0E0FA0709F0FC
:1001460048C0E1E0CE2EAA24BB2425E030E02530CD
:10015600E1E03E074CF4A0EEB0E0A20FB31FEC9135
:10016600F3D02F5F3F4FF3CFF501F070DF01E09141
:10017600E501F0E0EA17FB0749F4EB2DF070DF012B
:10018600E091E601F0E0EA17FB0709F01FC0949A38
:10019600959A969AEFEFE4BBDBD088249924E6D0B3
:1001A60078F4E9D0EED0E5BB979881E791E0019726
:1001B600F1F7979AE6D0C8D0F40131964F01EFCF08
:1001C600969895989498E2D0A9EC01C0AAEC65DFC0
:1001D60070C0E53CA0E0FA0719F5CC24D7D0949A74
:1001E6009798AA24BB24B4D0A9ECD4D0D3D0D2D02B
:1001F600D1D053DF88249924B9D050F4BCD003B3AE
:10020600E02FA2D0A02F49DFF40131964F01F4CFA1
:10021600EA2DAE2F42DFAB2D40DF979A949849C066
:10022600E63CA0E0FA0769F5CC24E0E8E2BBA0E0F2
:10023600B0E03ADFEFEFE4BBE5BB949A929AAFE009
:10024600B0E0ABD0959A969A9798A8E7B0E0A5D07B
:10025600979AAFE0B0E0A1D096989598929896D0EC
:1002660097986624772487D003B30F3F11F0AAEC42
:1002760004C0062C0728B9F7A9EC0FDF979A9498C3
:1002860018C0E73CA0E0FA0719F4CC24B6CE11C09A
:10029600E83CA0E0FA0769F4E1E0CE2EE091E10047
:1002A600E2BB56D0D30100DFEFEFE4BBE091E40000
:1002B600E5BBA1D02496E991EFBFF991E991B991F7
:1002C600A9919991899179916991F99019900990DB
:1002D6001895ECEFE1BBE0E8E2BBEFEFEABBE0E04C
:1002E600EBBBEFEFE7BBE0E0E8BB50D0E0E0E6B900
:1002F600E7B9E3BFE2BFE1BFEFBDEEBDEDBDECBDCB
:10030600E5BDE4BDEBBDEABDE9BDE8BDE9BFE5BFBE
:10031600E6BFEBB9E8E9EAB9E6E8E0BDE0E0E0BD52
:10032600E3E0E9B9E0E8E8B9E0E0EDB97894CC209B
:1003360041F4D394A8EEB3E030D0E2E0ED1509F431
:100346005CCEF5CF0000FECFF0E0AE0EBF1E0895E6
:10035600A091E200B0E0E0E0F1E035D0DF01E0910D
:10036600E100F0E0EA0FFB1F3F010895E0E0F1E055
:100376008E169F060895F30131963F013197DF01EE
:1003860093CEF401EB51FF4FE0810895E0E0E4BB2A
:10039600E5BB089582DEA0E00895109639F086E662
:1003A6009EE00197F1F7A8951197C9F70895F19581
:1003B600E195F0400895FA9FF02DEB9FF00DEA9F2E
:1003C600E02DF10D089504D0F6DF0EF4F0DF089568
:1003D600E894F7FF02C0EBDF6894B7FF06C0A0956C
:1003E600B095119600F8039400FA08953A932A936B
:1003F6001A930A9308953B812A81198108810895E9
:00000001FF
